:100000006EC0E6C187C086C085C084C083C082C080
:1000100081C080C07FC07EC07DC07CC07BC07AC0F4
:1000200079C078C077C00403090418037200610026
:10003000700068006E00650074002E006E006500A0
:1000400074001603470043002F004E0036003400B2
:100050005F0055005300420012011001000000082B
:1000600081179A0A0301010200010902220001011D
:100070000080320904000001030000000921010191
:1000800000012235000705810308000A0A03310038
:10009000300030003000120101010000000881171B
:1000A0009A0A03010102030105010905A1010901E1
:1000B000A100050109300931093309340935093630
:1000C000150026FF00750895068102C00509190173
:1000D000291015002501750195108102C000112419
:1000E0001FBECFE5D4E0DEBFCDBF10E0A0E6B0E09C
:1000F000E0EDF0E102C005900D92AE38B107D9F7FE
:1001000010E0AEE8B0E001C01D92A73FB107E1F7F3
:1001100005D3DCC775CF85B7826085BF8BB7806498
:100120008BBF8BE48093CD008AE58093CC0008954B
:100130001F93CF93DF939091DD00935097FDA2C062
:100140002091DA008091D9008D3209F099C0983061
:1001500009F096C0CCE0D0E0C21BD109CF51DF4FEF
:1001600083EC8093C1008AE58093600010928E003A
:100170008881807621F0CE018AD2282F78C09A819A
:100180001092CA008981882321F41092CB0022E0CA
:1001900068C0853019F49093DE0062C0863009F0A3
:1001A0004BC08B81813041F488E590E09093DC0076
:1001B0008093DB0022E13CC0823041F48AE690E08B
:1001C0009093DC008093DB0022E232C08330F9F4AC
:1001D0008A81882341F486E290E09093DC0080934A
:1001E000DB0024E025C0813041F48AE290E0909366
:1001F000DC008093DB0028E11BC08230C1F482E484
:1002000090E09093DC008093DB0026E111C0813206
:1002100041F48CE790E09093DC008093DB0029E0D0
:1002200007C0823221F4CE010DD2282F01C020E078
:1002300080E480938E001BC0883021F421E080EEA2
:1002400090E011C0893019F49093E00009C08A3021
:1002500011F421E006C08B3019F48BE48093CD00BB
:1002600020E08AEC90E09093DC008093DB008F81AB
:10027000882321F48E81821708F4282F20936100AF
:100280001092DD008091600084FF49C08091610080
:100290008F3F09F444C0182F893008F018E0811B03
:1002A000809361008091C10098E889278093C10004
:1002B000112341F12091DB003091DC0080918E0010
:1002C00086FF0DC0A2ECB0E080E090E0F901E80FFD
:1002D000F91FE491ED9301961817C1F708C0912F0B
:1002E000D901E2ECF0E08D9181939150E1F711504A
:1002F000812F90E01F5F0196820F931F9093DC0087
:100300008093DB0082EC90E0612F5ED0612F6C5F08
:100310006C3019F08FEF809361006093600094E17E
:1003200080B3857031F49150D9F71092DE001092AD
:10033000D800DF91CF911F9108951F93DC01162FF4
:100340008091CC0084FF07C08091CD0098E8892778
:100350008093CD0003C08AE58093CC00912FEEEC12
:10036000F0E08D91819391501916DCF38EEC90E0C2
:10037000612F2AD01C5F1093CC001F910895A82FE5
:10038000B92F8FEF9FEF1BC02D918227282F229529
:100390002827722F269526952727239526952170A5
:1003A000782F892F82272195207C922F22277695DE
:1003B000279597278227769527959727822761503B
:1003C00018F7809590950895DADF8D939D930895A1
:1003D000CF93CFB7CF93C395809BE9F7809B09C09C
:1003E000809B07C0809B05C0809B03C0809B01C091
:1003F000A3C0DF93C091DA00DD27CF51DF4F809B90
:1004000002C0DF91EBCF2F930F931F9300B32FEF19
:1004100000FB20F94F933F9310B34FEF012700FBF0
:1004200021F93BE031C04E7F012F10B3216028C07D
:10043000102F4D7F2260000000B329C04B7F246045
:10044000012F000010B32BC010B3477F28602AC0D3
:100450004F7E00B320612CC04F7D10B320622FC0AF
:100460004F7B00B3206432C0422700B349934FEF63
:100470000000102710FB20F910B31570C9F1297F77
:1004800091F2012700FB21F900B3237F89F231505B
:1004900058F1102710FB22F910B3277E79F20127BB
:1004A00000FB23F92F7C81F200B3102710FB24F905
:1004B0002F7971F200C010B3012700FB25F92F73CB
:1004C00059F200C000B3102710FB26F9223040F289
:1004D00000C010B3012700FB27F9243028F64F771E
:1004E000206810B30000F9CF10E41ABF002719C02C
:1004F0003B503195C31BD04010E41ABF0881033C28
:10050000F9F00B34E9F02091D8001981110F121382
:10051000EDCF4A81441F093641F10D3211F0013E01
:1005200029F70093DF003F914F911F910F912F9179
:10053000DF91CAB7C6FD4FCFCF91CFBFCF911895EE
:100540002091DF00222379F31091DD00112369F55A
:1005500034306AF13093DD002093D9001091DA0035
:100560003BE0311B3093DA0022C00091DD00013006
:10057000E4F40AE54F7049F43091600034FD19C08D
:1005800000936000C1ECD0E018C03091CC0034FD85
:1005900010C00093CC00CDECD0E00FC02795A8F49C
:1005A0005150A9F4220F0000F9CF4AE503C042EDF3
:1005B00001C0432FC4E1D0E032E011B31560909A3E
:1005C00011BB02B320E415E05F93012756E002BBA4
:1005D000279520F4515021F4220FF9CF012756E03E
:1005E00000003B5A02BBD0F2279528F4515029F461
:1005F000220F0000F9CF012756E0279502BB20F417
:10060000515021F4220FF9CF012756E029913323CD
:1006100002BB21F60A7F1091DE00110FC651D040B7
:1006200002BB11F01093D80010E41ABF016011B39F
:100630001A7F402F4A7F5F9100C000C002BB11BBF0
:1006400042BB71CFFC0180818076F9F481818630D4
:10065000E1F48381813019F08232B9F40BC08091CA
:100660009200909193009093DC008093DB00809146
:100670009400089580918F00909190009093DC00F9
:100680008093DB0080919100089580E00895FC0143
:1006900027E930E03093DC002093DB008081807616
:1006A0008032D1F58181813031F5E0919500F09172
:1006B00096003097A1F48FE780939700809398007D
:1006C0008093990080939A0080939B0080939C0074
:1006D00010929D0010929E0088E090E0089500889E
:1006E000F189E02DC9010995E0919500F0919600FE
:1006F000808191810895823041F48FE990E0909358
:10070000DC008093DB0081E008958A3029F4838146
:1007100080939F0080E0089580E00895AF92BF929B
:10072000CF92DF92EF92FF920F931F93CF93DF93BD
:1007300014BABB24BA94B5BA48EFC42EC2BA15E0B5
:1007400011BB38EEE32E30E8F32EC7010197F1F725
:1007500011BA13BF0FE005BD24ECD22ED3BC88EA3A
:1007600090E09093900080938F00A0D480939100AC
:1007700086E990E090939300809392000FD380934A
:10078000940014BAB5BAC2BA11BBC7010197F1F708
:1007900011BA13BF05BDD3BC88E190E00FB6F89441
:1007A000A89581BD0FBE01BDB6DC7894CC24BB24D6
:1007B000B394DD2400E010E090E8A92EFF24F39428
:1007C000CCE2D1E001C0DE2CA8950F31110524F058
:1007D000109296001092950080919500909196004D
:1007E000892B09F03CC0A4DCCBD2FC01909396008D
:1007F000809395000284F385E02D0995E0919500A2
:10080000F09196000288F389E02D0995882329F557
:1008100080E991E0FE013197F1F70197D9F788DC83
:1008200037D4FC0190939600809395000284F38561
:10083000E02D0995E0919500F09196000288F389EA
:10084000E02D0995882349F480E991E0FE01319774
:10085000F1F70197D9F76CDCB7CF00E010E0A8956D
:1008600067DCBB2089F0E0919500F091960004844C
:10087000F585E02D0995882321F4BB2400E010E0E4
:1008800003C00F5F1F4FBB2408B600FE0FC0F8BEA9
:10089000E0909F00EE2051F084E08D1518F0CC24FC
:1008A000C39405C08BEFE82EED0C01C0ED2C08B60B
:1008B00007FE20C0A8BECC2001F5E0919500F09184
:1008C00096000484F585E02D0995882319F400E04D
:1008D00010E002C00F5F1F4FE0919500F09196006D
:1008E0000684F785E02D0995882309F46CCFCC2484
:1008F000C39403C0CC2009F466CF8091CC0084FF60
:1009000062CFE0919500F09196000088F189E02D8A
:1009100087E990E00995E0919500F091960087E9CC
:1009200090E060810ADDDE2CCC244ECF009741F0B0
:10093000DC01E0EAF0E088E001900D928150E1F7FF
:10094000A8EAB0E0E0EAF0E088E001900D92815082
:10095000E1F708958091760090917700892B31F02E
:10096000109277001092760081E0089580EA90E07E
:1009700068EA70E048E050E09CD308950F931F931D
:10098000DF93CF93CDB7DEB7C954D0400FB6F894FC
:10099000DEBF0FBECDBF80E004D2BE01675F7F4FD8
:1009A00080E0FB01EF93FF9300E810E41023A9F02F
:1009B0000000A59A000000000000000000000000F8
:1009C0000000000000000000A59838E03A95F1F71B
:1009D00000000000069561F0E8CFA59A3BE03A954B
:1009E000F1F70000A59800000000069509F0DDCFA2
:1009F000A59800E813E01023A9F00000A59A0000D4
:100A000000000000000000000000000000000000E6
:100A10000000A59838E03A95F1F70000000006952F
:100A200061F0E8CFA59A3BE03A95F1F70000A59870
:100A300000000000069509F0DDCFA59800E8182F0A
:100A40001023A9F00000A59A00000000000000009B
:100A5000000000000000000000000000A59838E041
:100A60003A95F1F700000000069561F0E8CFA59AED
:100A70003BE03A95F1F70000A598000000000695CC
:100A800009F0DDCFA5980000000000000000A59A45
:100A90000000000000000000A59813B31072E9F3F5
:100AA00030E40FE30A9529F113B31072D9F7C19816
:100AB0000000000000000000000000000000000036
:100AC000000000000000000000000000000023B350
:100AD000C19A207221933A9539F00FE30A9549F0B3
:100AE00023B32072F1F6FACF882705C0C19A832F6D
:100AF00002C088278095FF91EF91C1988F3F21F424
:100B000081E08093B0001CC1FE01319688E0DF01D6
:100B10001D928A95E9F7498120E030E0DB0160E829
:100B200070E0F9017096EA0FFB1F8081882339F08D
:100B3000CB01022E02C0959587950A94E2F7482BC7
:100B40002F5F3F4F2830310561F749834A8120E00C
:100B500030E0DE01199660E870E0F9017896EA0F5E
:100B6000FB1F8081882339F0CB01022E02C09595AE
:100B700087950A94E2F7482B2F5F3F4F28303105C5
:100B800061F740954A834B8120E030E0DE01199601
:100B900060E870E0F901B096EA0FFB1F80818823BE
:100BA00039F0CB01022E02C0959587950A94E2F7A1
:100BB000482B2F5F3F4F2830310561F74B834C8125
:100BC00020E030E0DE01199660E870E0F901B896A7
:100BD000EA0FFB1F8081882311F080E007C0CB0162
:100BE000022E02C0959587950A94E2F7482B2F5F55
:100BF0003F4F2830310551F74C834D8120E030E0E4
:100C0000DE01199660E870E0F901F096EA0FFB1F2B
:100C10008081882339F0CB01022E02C095958795FB
:100C20000A94E2F7482B2F5F3F4F2830310561F7D8
:100C300040954D834E8120E030E0DE01199660E85A
:100C400070E0F901F896EA0FFB1F8081882339F0E4
:100C5000CB01022E02C0959587950A94E2F7482BA6
:100C60002F5F3F4F2830310561F740954E834F810C
:100C700020E030E0DE01199661E070E0F901339682
:100C8000EA0FFB1F8081882339F0CB01022E02C0BE
:100C9000880F991F0A94E2F7482B2F5F3F4F2530AA
:100CA000310561F720E030E0DE01199660E270E086
:100CB000F9013996EA0FFB1F8081882339F0CB01B7
:100CC000022E02C0880F991F0A94E2F7482B2F5F6B
:100CD0003F4F2330310561F74F83488520E030E0F6
:100CE000DE01199661E070E0F9013C96EA0FFB1F06
:100CF0008081882339F0CB01022E02C0880F991F12
:100D00000A94E2F7482B2F5F3F4F2430310561F7FB
:100D100089818093A0008A818093A1008B81809338
:100D2000A2008C818093A3008D818093A4008E818A
:100D30008093A5008F818093A6004093A70080E058
:100D4000C75BDF4F0FB6F894DEBF0FBECDBFCF91AC
:100D5000DF911F910F9108951092B0000FDE90E087
:100D60008091B000882309F491E0892F08958FB70E
:100D7000F894B99AC198A598AD988FBFFFDD0895F2
:100D800088EA90E090936700809366008FD19093FB
:100D900065008093640082E690E0089582E190E02F
:100DA00008950F931F93DF93CF93CDB7DEB7C05055
:100DB000D1400FB6F894DEBF0FBECDBF00E8182FAC
:100DC0001023A9F00000A59A000000000000000018
:100DD000000000000000000000000000A59828E0CE
:100DE0002A95F1F700000000069561F0E8CFA59A7A
:100DF0002BE02A95F1F70000A59800000000069569
:100E000009F0DDCFA5980000000000000000000000
:100E10000000000000000000A59A00000000000093
:100E20000000A5980FEF0A9511F09D9BFCCFFE01E5
:100E30003196EF93FF93882700270395B1F09D9992
:100E4000FCCFC19808C00027039579F09D99FCCF8D
:100E5000839551F001930027039539F09D9BFCCFBA
:100E6000839511F00193EFCFC19AFF91EF918134F7
:100E700019F02FEF3FEFAFC09F01BE016F5B7F4FB7
:100E800040E090818181981708F441E0D9014D93A9
:100E90009D013296E617F70799F720E030E010E061
:100EA000BE016F5F7F4F41E050E0FB01E20FF31F97
:100EB0008081882339F0CA01022E02C0880F991F51
:100EC0000A94E2F7182B2F5F3F4F2430310569F762
:100ED000FE013D9620E030E040E150E08081882333
:100EE00039F0CA01022E02C0880F991F0A94E2F756
:100EF000182B2F5F3F4F31962430310579F79B85B2
:100F0000911191E08C85811182E0682F692BFE019F
:100F1000719620E030E050E0A0E8B0E080818823C6
:100F200039F0CD01022E02C0959587950A94E2F71B
:100F3000582B2F5F3F4F31962830310579F7FE014E
:100F4000799620E030E040E0A0E8B0E0808188239E
:100F500039F0CD01022E02C0959587950A94E2F7EB
:100F6000482B2F5F3F4F31962830310579F7515884
:100F70005093B1008FE7982F941B9093B200809309
:100F8000B3008093B4008093B5008093B6001093B3
:100F9000B7006093B8008D81882319F06460609376
:100FA000B8008E81882329F08091B80088608093F2
:100FB000B8008F81882329F08091B80080618093E8
:100FC000B8008885882329F08091B80080628093DA
:100FD000B80020E030E0C901C050DF4F0FB6F894F0
:100FE000DEBF0FBECDBFCF91DF911F910F9108954E
:100FF00081E0D7DE08958FB7F894B99AC198A59883
:10100000AD988FBFF5DF08951F93CF93DF9310E066
:10101000CCE2D1E00DC0FE013197F1F70197D9F78D
:10102000E7DF882341F01F5F1F3011F480E004C028
:101030008CE291E0F0CF81E0DF91CF911F91089594
:10104000009741F0DC01E1EBF0E088E001900D92C7
:101050008150E1F7A9EBB0E0E1EBF0E088E001902E
:101060000D928150E1F7089580918C0090918D0050
:10107000892B31F010928D0010928C0081E0089540
:1010800081EB90E069EB70E048E050E012D0089509
:1010900088EA90E090937D0080937C0007D0909345
:1010A0007B0080937A0088E790E0089585E390E0E4
:1010B0000895FB01DC0104C08D910190801921F499
:1010C00041505040C8F7881B990B0895F894FFCF02
:1010D0005AFF08000000000000000000B706BE0430
:1010E000AA049604AC0601000800000000000000FD
:0E10F0000000FB07F807340820080408010080
:00000001FF
